:100000000C945C000C94D5010C9402020C948400B6
:100010000C9484000C9484000C9484000C94840050
:100020000C9484000C9484000C9484000C94840040
:100030000C9484000C9484000C9484000C94840030
:100040000C942F020C9484000C941A040C948400D9
:100050000C9484000C9484000C9484000C94840010
:100060000C9484000C948400000024272A000025AE
:10007000282B000023262904040404040404040299
:100080000202020202030303030303010204081035
:100090002040800102040810200102040810200002
:1000A0000000070002010000030406000000000039
:1000B000000000008600CA0111241FBECFEFD4E06B
:1000C000DEBFCDBF11E0A0E0B1E0ECE0F9E002C09E
:1000D00005900D92A831B107D9F711E0A8E1B1E080
:1000E00001C01D92AA3BB107E1F710E0C8EBD0E0D8
:1000F00004C02297FE010E948004C43BD107C9F7C7
:100100000E94C3010C9484040C94000080910001AF
:100110009091010190931F0180931E0108950F9308
:100120001F93809106010E94C603892B09F0D4C059
:100130008091180190911901892B09F0CDC020916F
:100140000E0130910F0180910C0190910D01280F4B
:10015000391F2F3F31053CF08FEF90E090930D0158
:1001600080930C0104C030930D0120930C0181E0B9
:1001700090E0909319018093180104C01092190126
:1001800010921801809108010E94C603892B09F082
:10019000ABC080911A0190911B01892B09F0A4C07A
:1001A00086E990E090930D0180930C0181E090E04E
:1001B00090931B0180931A0104C010921B011092AE
:1001C0001A0180910A010E94C603892B09F094C08C
:1001D00080911C0190911D01892B09F08DC08091A7
:1001E0000C0190910D0120910E0130910F01281703
:1001F00039072CF010920D0110920C0106C0821BE1
:10020000930B90930D0180930C0181E090E090930B
:100210001D0180931C0104C010921D0110921C014D
:1002200060910C0170910D01809104010E94050301
:1002300081E00E94E7028C0180E00E94E7028017C3
:1002400091070CF061C080911E0190911F012091D7
:10025000220130912301821B930B209100013091E8
:100260000101281739070CF44FC061E080910201A9
:100270000E947B030E949F0270931F0160931E01E6
:100280004EC00E949F02709323016093220160E0A0
:10029000809102010E947B0380911E0190911F01B9
:1002A00090932101809320013AC080911E0190918A
:1002B0001F012091220130912301821B930B209179
:1002C000000130910101281739074CF560E0809159
:1002D00002010E947B0323C0809106010E94C60395
:1002E000019709F04FCF4ACF809108010E94C603C1
:1002F000019709F066CF61CF80910A010E94C60381
:10030000019709F08DCF88CF81E00E94E7028C0130
:1003100080E00E94E702081719073CF6B2CF1F9150
:100320000F91089561E0809102010E945D0360E0F9
:10033000809106010E945D0360E0809108010E94A7
:100340005D0360E080910A010E945D0361E08DE041
:100350000E945D0361E0809104010E945D0361E001
:10036000809106010E947B0361E0809108010E9458
:100370007B0361E080910A010E947B0361E08DE0D4
:100380000E947B0308950E94AD020E9492010E9488
:100390008F00FDCF85E191E09093250180932401AA
:1003A0000895862F0E94120408951F920F920FB68F
:1003B0000F9211242F933F934F935F936F937F93EB
:1003C0008F939F93AF93BF93EF93FF9380912601F9
:1003D00090912701892B29F0E0912601F0912701C6
:1003E0000995FF91EF91BF91AF919F918F917F916F
:1003F0006F915F914F913F912F910F900FBE0F9092
:100400001F9018951F920F920FB60F9211242F93E1
:100410003F934F935F936F937F938F939F93AF938C
:10042000BF93EF93FF938091280190912901892B2D
:1004300029F0E0912801F09129010995FF91EF91B0
:10044000BF91AF919F918F917F916F915F914F91EC
:100450003F912F910F900FBE0F901F9018951F92F4
:100460000F920FB60F9211242F938F939F93AF93F8
:10047000BF9380912A0190912B01A0912C01B09102
:100480002D010196A11DB11D80932A0190932B018E
:10049000A0932C01B0932D0180912E0190912F01FA
:1004A000A0913001B09131018050904CAF4FBF4FBF
:1004B00080932E0190932F01A0933001B0933101CE
:1004C00027C080912E0190912F01A0913001B09111
:1004D000310180589E43A040B04080932E019093FC
:1004E0002F01A0933001B09331018091320190919E
:1004F0003301A0913401B09135010196A11DB11DC8
:100500008093320190933301A0933401B09335016D
:1005100080912E0190912F01A0913001B091310175
:1005200081589E43A040B04060F6BF91AF919F912B
:100530008F912F910F900FBE0F901F9018958FB72E
:10054000F89420913201309133014091340150915F
:1005500035018FBFB901CA010895789484B58260CE
:1005600084BD84B5816084BD85B5826085BD85B557
:10057000816085BDEEE6F0E0808181608083E1E806
:10058000F0E0808182608083808181608083E0E808
:10059000F0E0808181608083E1EBF0E08081846025
:1005A0008083E0EBF0E0808181608083EAE7F0E027
:1005B000808184608083808182608083808181608B
:1005C00080838081806880831092C10008958F703D
:1005D000909110019295990F990F907C982B909380
:1005E0007C0080917A00806480937A0080917A0008
:1005F00086FDFCCF2091780040917900942F80E017
:1006000030E0282B392BC90108951F93CF93DF9336
:10061000182FEB0161E00E945D03E12FF0E0E1564D
:10062000FF4F8491833051F48091800080688093E3
:100630008000D0938900C09388003BC0843051F47F
:1006400080918000806280938000D0938B00C09363
:100650008A002FC0813039F4209729F184B5806851
:1006600084BDC7BD26C0823039F42097E1F084B53F
:10067000806284BDC8BD1DC0863041F48091B00049
:1006800080688093B000C093B30013C0873041F4FA
:100690008091B00080628093B000C093B40009C024
:1006A000C038D10514F460E001C061E0812F0E94E0
:1006B0007B03DF91CF911F910895282F30E0C9016E
:1006C00085579F4FFC01949129583F4FF901849120
:1006D000882381F0E82FF0E0E859FF4FE491F0E043
:1006E000662329F4808190958923808308958081F1
:1006F000892B80830895482F50E0CA0181569F4F6F
:10070000FC012491CA0185579F4FFC0194914958DF
:100710005F4FFA0134913323C1F1222331F12330A9
:1007200021F4809180008F7705C0243031F48091CE
:1007300080008F7D8093800018C0213019F484B52B
:100740008F7704C0223021F484B58F7D84BD0DC025
:10075000263021F48091B0008F7705C0273029F42E
:100760008091B0008F7D8093B000E32FF0E0E359DB
:10077000FF4FE491F0E0662329F48081909589236E
:10078000808308958081892B80830895482F50E0CD
:10079000CA0181569F4FFC012491CA0185579F4F82
:1007A000FC01949149585F4FFA013491332319F4B5
:1007B00020E030E035C0222331F1233021F4809154
:1007C00080008F7705C0243031F4809180008F7DC8
:1007D0008093800018C0213019F484B58F7704C04D
:1007E000223021F484B58F7D84BD0DC0263021F4E4
:1007F0008091B0008F7705C0273029F48091B00038
:100800008F7D8093B000E32FF0E0EE58FF4FE4912E
:10081000F0E0808120E030E0892311F021E030E039
:10082000C9010895982F8091C00085FFFCCF909357
:10083000C60008951F920F920FB60F9211242F93A6
:100840003F934F935F936F937F938F939F93AF9358
:10085000BF93EF93FF934091C600E0913601F09172
:100860003701CF01019660E870E00E9457049C01B7
:1008700080913801909139012817390739F0E65CE9
:10088000FE4F40833093370120933601FF91EF9163
:10089000BF91AF919F918F917F916F915F914F9198
:1008A0003F912F910F900FBE0F901F90189597FBBF
:1008B000092E07260AD077FD04D00CD006D00020E0
:1008C0001AF4709561957F4F0895F6F7909581958C
:1008D0009F4F0895AA1BBB1B51E107C0AA1FBB1F56
:1008E000A617B70710F0A61BB70B881F991F5A95BC
:1008F000A9F780959095BC01CD010895EE0FFF1FDB
:0C0900000590F491E02D0994F894FFCFCD
:10090C00050002000900110012001300FF00010095
:08091C000100000000D1010000
:00000001FF
